:1000000000308A00A72C0000FF00030E8301A1002E
:100010000A08A0008A010408A2007708A300780853
:10002000A4007908A5007A08A6007B08A70083131E
:1000300083128C308400001D1F280C1932282208DE
:1000400084002308F7002408F8002508F900260892
:10005000FA002708FB0020088A00210E8300FF0E0B
:100060007F0E09008A110A1235281430AB0083165E
:100070000814831208183F285030AE004928831610
:1000800008158312081947285F30AE00492801304F
:10009000AE00831688158312881951285030AF009E
:1000A0005B28831688148312881859285F30AF00A4
:1000B0005B280130AF000C118A110A121F283F3053
:1000C00085008601FF308700880189012030831672
:1000D0008500FF3086001F3087008312DC00FF3070
:1000E00083168800091089100911811383121F08D3
:1000F00038399F00063083169F0083129412DC1259
:100100005C088316870083125C165C0883168700E0
:1001100085168312DC155C08831687003430831241
:100120009400003083169400831207119701053064
:10013000970083160C15C03083128B04A801A90107
:10014000AA011430AB000130AE000130AF008A11BB
:100150000A12B12C0830F700F70BAC2883160512F1
:10016000831205120330F700F70BB4288316051627
:10017000831200345C155C0883168700831207190C
:10018000BA28AB012B08033C031C1329831614184F
:10019000CB288312C62883121308AC0094131413BF
:1001A0002B08F700F7080319E2280130770203193A
:1001B000EB28023077020319EE2803307702031987
:1001C000F22801294230AD002C08803C0319EA28AE
:1001D0001430AB0004295A30AD00042908086038F7
:1001E000AD0004290608AD003108C23C031D0029FA
:1001F0002C08803C031D00290230A8001430AB00FD
:100200000429FF30AD0004292D08930030302B075E
:1002100084002C08800046302B0784002D088000C5
:10022000AA20AB0AC2288A110A12C42C5C155C08E9
:1002300083168700831207191629AB012B08073C88
:10024000031C872983161418272983122229831255
:100250001308AC00941314132B08F700F7080319C4
:100260004E2901307702031957290230770203190A
:100270005A290330770203195E29043077020319E3
:1002800061290530770203196429063077020319C2
:1002900067290730770203196A297529CE30AD0026
:1002A0002C08803C031956291430AB0078295A30A9
:1002B000AD00782908086F38AD0078290608AD0030
:1002C00078290130AD0078290130AD0078292E0859
:1002D000AD0078292F08AD003108C23C031D7429F8
:1002E0000230A8001430AB007829FF30AD00782927
:1002F0002D08930030302B0784002C0880004630F6
:100300002B0784002D088000AA20AB0A1E298A1121
:100310000A12C62C02302B02FA3E0318A729063E09
:10032000AA29C030AD00A7294030AD00A729A908EF
:10033000031D9C29AD019E298030AD00A7294030C6
:10034000AD00A7298030AD00A729AD01A7298A11EA
:100350000A12BD2B0A148A100A11820791299429C6
:1003600097299F29A229A52902302B02FA3E0318BA
:10037000DC29063EDF29AD01DC29AD01DC29803016
:10038000AD00DC29B308031DC8294030AD00CA29DF
:100390008030AD00DC29B308031DD029AD01D2297E
:1003A0008030AD00DC29B308031DD9295030AD00E1
:1003B000DB292830AD00DC298A110A12BF2B0A1470
:1003C0008A100A118207BB29BD29BF29C229CB295E
:1003D000D32902302B02FA3E0318FE29063E012AD9
:1003E000AD01FE29AD01FE294030AD00FE29AD0171
:1003F000FE298030AD00FE29AD01FE298A110A12C6
:10040000C12B0A108A140A118207F029F229F42953
:10041000F729F929FC2902302B02FA3E0318252A74
:10042000063E282AAD01252AAD01252AAD01252A3F
:10043000B308031D1E2A2030AD00202AE030AD0095
:10044000252AAD01252AAD01252A8A110A12C32BBE
:100450000A108A140A118207122A142A162A182A44
:10046000212A232A02302B02FA3E0318562A063E7E
:10047000642AAA08031D3F2AFF30AD00402AAD01BF
:10048000562AAA08031D472AFF30AD00492A8030AA
:10049000AD00562AFF30AD00562AFF30AD00562A77
:1004A000FF30AD00562AFF30AD00562AB308031DB9
:1004B000602A3408803C031D602A0130AA00612AAA
:1004C000AA018A110A12C52B0A108A140A1182077E
:1004D000392A412A4A2A4D2A502A532AA908031D9B
:1004E000852A02302B02FA3E0318842A063EA62AE9
:1004F000AD01842AAD01842AAD01842AAD01842A8C
:10050000AD01842AAD01842AA32A290B882A8C2ACA
:100510002908023C031DA32A02302B02FA3E0318CD
:10052000A32A063EB02AFF30AD00A32AFF30AD005B
:10053000A32AC030AD00A32AAD01A32AAD01A32A8E
:100540005A30AD00A32A8A110A12C72B0A108A1446
:100550000A118207782A7A2A7C2A7E2A802A822A0D
:100560000A108A140A118207932A962A992A9C2A29
:100570009E2AA02A02302B02FA3E0318CD2A063EFC
:10058000E12AAD01CD2AAD01CD2AAD01CD2AAD01C3
:10059000CD2AAD01CD2AAD01CD2AB308031DDE2A37
:1005A0002908FD3E0318DE2A033EEB2AA801DE2AB5
:1005B0000130A800DE2A0330A800DE2A8A110A12C0
:1005C000C92B0A108A140A118207C12AC32AC52A14
:1005D000C72AC92ACB2A0A108A140A118207D62AE6
:1005E000D82ADB2A02302B02FA3E0318052B063EDE
:1005F000132BAD01052BAD01052BAD01052BAD0175
:10060000052BAD01052BAD01052B3308803C031DE7
:100610000C2B0130A900102BB308031D102BA901CE
:100620008A110A12CB2B0A148A140A118207F92A9A
:10063000FB2AFD2AFF2A012B032B02302B02FA3E54
:100640000318312B063E362BAD01312BAD01312B7A
:10065000AD01312BAD01312BAD01312B5A30AD0045
:10066000312B0230A9008A110A12CD2B0A148A14E8
:100670000A118207242B262B282B2A2B2C2B2E2BDE
:1006800002302B02FA3E0318552B063E582BAD01C3
:10069000552BAD01552B4030AD00552BAD01552BE1
:1006A000AD01552B5A30AD00552B8A110A12CF2BB4
:1006B0000A148A140A118207472B492B4B2B4E2B05
:1006C000502B522B5C155C08831687008312071988
:1006D000622BAB012B08073C031CE52B8316141877
:1006E000732B83126E2B83121308AC009413141314
:1006F000AB08031D842BCF30AD002C08803C0319C0
:10070000832B1430AB00D62B2B0B892B5A30AD002A
:10071000D62B2B08013C0318D42B2B08073C031CB9
:10072000D42B3108F700A23077020319BC2B6230BA
:1007300077020319BE2BE23077020319C02B323047
:1007400077020319C22BB23077020319C42B82300F
:1007500077020319C62BC23077020319C82B223047
:1007600077020319CA2BF23077020319CC2B02301F
:1007700077020319CE2BD02B8A29D32BB429D32B64
:10078000E929D32B0B2AD32B322AD32B6E2AD32B36
:10079000BA2AD32BF22AD32B1D2BD32B402BD32BAE
:1007A000FF30AD00D32BD62B1430AB002D089300B7
:1007B00030302B0784002C08800046302B07840043
:1007C0002D088000AA20AB0A6A2B8A110A12C82CB5
:1007D0005C155C088316870083120719E82BAB01B0
:1007E0002B08133C031CA42C83161418F92B83121A
:1007F000F42B83121308AC00941314132B08F70086
:10080000F7080319502C013077020319592C0230D4
:10081000770203195C2C033077020319602C043033
:1008200077020319622C053077020319652C063014
:1008300077020319682C0730770203196B2C0830F4
:10084000770203196E2C093077020319702C0A30D5
:1008500077020319722C0B3077020319742C0C30B9
:1008600077020319762C0D3077020319782C0E309D
:10087000770203197A2C0F30770203197C2C103081
:10088000770203197E2C113077020319802C123065
:1008900077020319822C133077020319842C922CCF
:1008A0009E30AD002C08803C0319582C1430AB004E
:1008B000952C5A30AD00952C08086038AD00952C69
:1008C0000608AD000130AD00952C0130AD00952C2F
:1008D0000130AD00952C0130AD00952CAD01952C6B
:1008E000AD01952CAD01952CAD01952CAD01952C4C
:1008F000AD01952CAD01952CAD01952CAD01952C3C
:10090000AD01952CAD01952CAD013108C23C031D04
:10091000912C3308803C031D912C0230A800143028
:10092000AB00952CFF30AD00952C2D089300303096
:100930002B0784002C08800046302B0784002D08EC
:100940008000AA20AB0AF02B8A110A12CA2C84015B
:100950001F308305073083169F00FF308312DC00B1
:100960005F282808F700F7080319C32C0130770225
:100970000319C52C023077020319C72C0330770204
:100980000319C92CCB2CBA28CC2C1629CC2C622BC1
:0C099000CC2CE82BCC2CCC2CB12C630020
:02400E00723FFF
:00000001FF
